:020000040000FA
:06000000CEEF06F0120035
:06080000CEEF06F012002D
:06082A000100D00D0000EA
:0808300000020000200000009E
:08083800D9CFE6FFE1CFD9FFA3
:10084000040EE126DE6ADE6ADE6ADD6ADD52DD5212
:10085000FD0EDBCF00F0FE0EDBCF01F0026A036A73
:1008600001AE02D002680368D9CFE9FFDACFEAFF10
:10087000030EEB500318E8AE02D0033408D000504A
:10088000EE5C0150EE580250EE580350EE580FE265
:100890000C0EE66EAEEC06F0E552D9CFE9FFDACFEA
:1008A000EAFFEE2A000EEE22EE22EE22D1D7040E4F
:1008B000E15C02E2E16AE552E16EE552E7CFD9FF81
:1008C00012000F0EC16E070EB46E936A816A300E6D
:1008D000926E80900F0E946EF19E1200D9CFE6FFBB
:1008E000E1CFD9FF020EE1268250020B01E0010E9A
:1008F000080DF3CF02F08250010B040DF3CF01F08D
:100900008050200B01E0010EE824006E8050100B97
:1009100001E0010E002401240224DE6EDD6ADECF38
:1009200000F0DDCF01F000C0F3FF01C0F4FF020EC4
:10093000E15C03E200D0E16AE552E16EE552E7CF07
:10094000D9FF12008092320EE66EDCEC06F0E55222
:100950008084320EE66EDCEC06F0E5528094320EB6
:10096000E66EDCEC06F0E55212008082010EE66EC7
:10097000E66A62DFE552E5528084010EE66EE66AC1
:100980005BDFE552E5528094010EE66EE66A54DFC5
:10099000E552E5521200380E816ED4DF320EE66E5B
:1009A000E66A4ADFE552E552010E816ECBDF320E78
:1009B000E66EE66A41DFE552E5520D0E816EC2DF5A
:1009C000320EE66EE66A38DFE552E552060E816EBB
:1009D000B9DF320EE66EE66A2FDFE552E55212000D
:1009E000010E816EAFDF0A0EE66EE66A25DFE55284
:1009F000E5521200D9CFE6FFE1CFD9FF020E816E9A
:100A0000A1DF0A0EE66EE66A17DFE552E552FD0E3B
:100A1000DBCFE6FFFE0EDB50280DF350E552E72456
:100A2000E76EFE0EE7CFDBFFFD0EDB6AFE0EDB504E
:100A3000F36EFD0EDBCFF4FFF350F45C0BE2140E0B
:100A4000816E80DF320EE66EDCEC06F0E552FD0EC4
:100A5000DB2AECD7E552E7CFD9FF1200D9CFE6FF6A
:100A6000E1CFD9FFFE0EDB50816E7FDF010EE66E17
:100A7000E66AE2DEE552E552E552E7CFD9FF120021
:100A8000D9CFE6FFE1CFD9FFFD0EDBCFE9FFFE0EA8
:100A9000DBCFEAFFEF500EE0FD0EDBCFE9FFDB2AF4
:100AA000FE0EDBCFEAFF01E3DB2AEF50E66ED6DF76
:100AB000E552EAD7E552E7CFD9FF12000201246BD5
:100AC000300E926EF00E936EEF0E206F20C281FFFB
:100AD000040E216F2151000821E22051FE0BE84253
:100AE000206F20C281FF050EE66EE66AA5DEE552A4
:100AF000E5528150100B09E08150200B06E0815037
:100B0000400B03E08150800B01E10AD8020124056B
:100B100002E1255104D02105216FDCD7CFD7120087
:100B2000F00E936E81CF23F202012315226F0F0E78
:100B30002015206F20512211206F81CF23F2F00E5B
:100B40002315226FF00E225D01E0F7D7936A06D8D5
:100B500026C225F20201010E246F12000201276B4A
:100B6000100E275D14E22751EA6A000FE96E020EAB
:100B7000EA22EF50205D08E12751EA6A100FE96E82
:100B8000020EEA22EFCF26F22729276FE9D726C2E5
:100B900081FF640EE66EE66A4FDEE552E552120012
:100BA0000201286B070E285D1DE288DF0201296F14
:100BB0002851EA6A2A0FE96E020EEA2229C2EFFFE3
:100BC0002851EA6A2A0FE96E020EEA22EF5046081F
:100BD00002E108D004D029C2E6FF40DFE55202015D
:100BE000282BE0D72851EA6A2A0FE96E020EEA2282
:100BF000EF6A12000201286B070E285D16E22851E9
:100C0000EA6A2A0FE96E020EEA22EF50E66E26DF4C
:100C1000E55202012829EA6A2A0FE96E020EEA2249
:100C2000EF5001E102D0282BE7D71200D9CFE6FF21
:100C3000E1CFD9FFE652F250800B01E0010EDF6EEA
:100C4000F29EA69EA69CA684FE0EDB50A96EFD0E0B
:100C5000DB50A86E550EA76EAA0EA76EA682A6B28E
:100C6000FED7A694DF50E8B0F28EE8A0F29EE552DF
:100C7000E552E7CFD9FF1200D9CFE6FFE1CFD9FF88
:100C8000A69CA69EFE0EDB50A96EA680A85000D0A2
:100C9000E552E7CFD9FF120014DE8180F40EE66E34
:100CA000010EE66EC9DDE552E5528190F40EE66E66
:0E0CB000010EE66EC1DDE552E552EED71200F0
:020CBE002A0EFC
:100CC000F66E080EF76E000EF86E02010900F55080
:100CD000386F0900F550396F03E1386701D03DD016
:100CE0000900F550336F0900F550346F0900F550D5
:100CF000356F09000900F550E96E0900F550EA6EFC
:100D0000090009000900F550366F0900F550376FEA
:100D100009000900F6CF3AF2F7CF3BF2F8CF3CF2E8
:100D200033C2F6FF34C2F7FF35C2F8FF0201365373
:100D300002E1375307E00900F550EE6E3607F8E29E
:100D40003707F9D73AC2F6FF3BC2F7FF3CC2F8FFBC
:0C0D500002013807000E395BBFD712000B
:040D5C00FF0EE35053
:100D6000066E480E01D04C0EE76EE72EFED7E76AFE
:0C0D7000E72EFED7062EF7D70000120079
:040D7C00000EF36E04
:100D800000EE00F0080E01D81200EA6002D0EE6A10
:0C0D9000FCD7F350E9601200EE6AFCD7BB
:040D9C0012EE40F023
:100DA00022EE40F0F86A059C5FEC06F0E7EC06F0F6
:080DB0004CEC06F0FBD7120029
:080DB800FF0EE350E84E1200AB
:0E0DC000000000D000D000D0E82EFAD71200BC
:020DCE00120011
:100DD000EEEDEBE7DEDDDBD7BEBDBBB77E7D7B771F
:100DE0003031323334353637383941424344454661
:00000001FF
